:1000000000308A0004280000FF238316900000308F
:100010008A008729353084008313000803192128BA
:100020000130A100BF30A0006400A00B1428A10B78
:1000300012284A30A000A00B1B2800006400800B8F
:100040001028003434080739A000340CA100A10C9A
:10005000A10C1F30A105210836078400831337182F
:100060008317A101A10AA00A3628A10DA00B3528EB
:10007000B50803193E28210880044128A109210858
:100080008005003434080739A000340CA100A10C0D
:10009000A10C1F30A10521083507840083133618F1
:1000A00083170008A100A00A5628A10CA00B552810
:1000B0000034B201B301A6013108260203188B28CF
:1000C0002F08B4000130B500B701B60122202F0877
:1000D000B400B501B7018030B60022200230B40070
:1000E000FA30B5000A20B40B70282F08B400B5010F
:1000F000B701B60122202F08B400B501B701803046
:10010000B60022200230B400FA30B5000A20B40B49
:100110008428A60A5C28B30132081D3C031CB928B8
:10012000B20A6430B5000A202D08B4000130B500D1
:10013000B7018030B60022202D08B400B601B50109
:1001400042202118B8282D08B4000130B500B701AD
:100150008030B60022202D08B400B601B50142203F
:100160002118B6286430B5000A20A328B201B30ACA
:100170008C283308A1000034831685158312851955
:10018000D02883160510831205143230B5000A20DA
:1001900083160510831205103230B5000A20BC28E2
:1001A0000430AD00FA30B5000A20AD0BD228AE0104
:1001B0002B30AD00B0012830AF000530B100592020
:1001C0002108A800AE012B30AD00B0012830AF00EF
:1001D0000430B10059202108A900AE012B30AD0038
:1001E000B0012830AF000330B10059202108AA0027
:1001F000AE012B30AD00B0012830AF000230B100AD
:1002000059202108AB00AE012B30AD00B0012830E1
:10021000AF000130B10059202108AC0083169B01CA
:100220008312280883169A001C1583120B08A0005D
:100230008B13831655309D00AA309D009C149C188A
:100240001F291C11831220088B04013083169B0088
:100250008312290883169A001C1583120B08A0002C
:100260008B13831655309D00AA309D009C149C185A
:1002700037291C11831220088B04023083169B003F
:1002800083122A0883169A001C1583120B08A000FB
:100290008B13831655309D00AA309D009C149C182A
:1002A0004F291C11831220088B04033083169B00F6
:1002B00083122B0883169A001C1583120B08A000CA
:1002C0008B13831655309D00AA309D009C149C18FA
:1002D00067291C11831220088B04043083169B00AD
:1002E00083122C0883169A001C1583120B08A00099
:1002F0008B13831655309D00AA309D009C149C18CA
:100300007F291C11831220088B0485291A2A840155
:1003100083131F3083051F1383161F109F101F1197
:100320009F110730831299000530A800A900AA0088
:10033000AB00AC001F1383161F109F101F119F11DD
:1003400083121F1083160108C739083881000C304A
:100350008312A000073081018130840083130008DC
:10036000F0390738800064000008F739A019F03927
:10037000200480009001073099008316050864006E
:1003800002308312A000A00BC329C62919088C11C2
:100390008316990105118312051183160510831226
:1003A00005140430AD00FA30B5000A20AD0BD32996
:1003B000831605108312051083169B019C131C14D1
:1003C0001A088312A800013083169B009C131C148A
:1003D0001A088312A900023083169B009C131C1478
:1003E0001A088312AA00033083169B009C131C1466
:1003F0001A088312AB00043083169B009C131C1454
:100400001A088312AC00A501831685158312851D79
:100410000D2A0130B5000A20042A8316851583129F
:1004200085191B2AA50A6430B5000A202508323C2C
:10043000031CBC280D2AA8080319302A83160511AD
:1004400083120515A601280826020318302A043055
:10045000AD00FA30B5000A20AD0B292AA60A232ADE
:10046000A90803194F2AA6012908260203184F2AB2
:10047000A7012708C73C031C4D2A831605118312C8
:1004800005150430B5000A208316051183120511E5
:100490000130B5000A20A70A392AA60A342AAA0878
:1004A00003196E2AA6012A08260203186E2AA7013C
:1004B0002708C73C031C6C2A8316051183120515F7
:1004C0000330B5000A20831605118312051102308E
:1004D000B5000A20A70A582AA60A532AAB0803190E
:1004E0008D2AA6012B08260203188D2AA7012708AA
:1004F000C73C031C8B2A8316051183120515023095
:10050000B5000A2083160511831205110330B500CA
:100510000A20A70A772AA60A722AAC080319AC2A6D
:10052000A6012C0826020318AC2AA7012708C73CFD
:10053000031CAA2A83160511831205150130B50084
:100540000A2083160511831205110430B5000A2014
:0C055000A70A962AA60A912A032A630033
:02400E004C3133
:00000001FF
